:100000000C9444000C946C000C946C000C946C00E8
:100010000C946C000C946C000C946C000C946C00B0
:100020000C946C000C946C000C946C000C946E009E
:100030000C946C000C946C000C946C000C946C0090
:100040000C946C000C946C000C94D9030C946C0010
:100050000C946C000C946C000C946C000C946C0070
:100060000C946C000C946C0005A84CCDB2D44EB925
:100070003836A9020C50B9918688083CA6AAAA2A4B
:10008000BE000000803FB70111241FBECFEFD8E0B3
:10009000DEBFCDBF11E0A0E0B1E0EEE7F6E102C0C7
:1000A00005900D92A232B107D9F713E0A2E2B1E0B8
:1000B00001C01D92AC3AB107E1F710E0C8E8D0E00A
:1000C00004C02297FE010E94A409C638D107C9F7CF
:1000D0000E945C010C943D0B0C9400001F920F9247
:1000E0000FB60F9211242F933F934F935F936F930B
:1000F0007F938F939F93AF93BF93EF93FF93DF9380
:10010000CF9300D0CDB7DEB7A5E2B0E0E5E2F0E0F6
:10011000908180E289278C931A82198220C0809175
:10012000240390912503FC01EE5DFE4F208186E2C1
:1001300093E0622F0E94BE018091240390912503D9
:10014000019620E032E0B9010E940709909325034F
:100150008093240389819A8101969A838983898176
:100160009A8121E080349207D4F286E293E060E045
:100170000E94BE010F900F90CF91DF91FF91EF9100
:10018000BF91AF919F918F917F916F915F914F91AF
:100190003F912F910F900FBE0F901F901895DF93F6
:1001A000CF93CDB7DEB764970FB6F894DEBF0FBE1E
:1001B000CDBF88ED9FE0A9E4B0E4898B9A8BAB8B2F
:1001C000BC8B80E090E0A0E0B0E08D879E87AF8799
:1001D000B88B29893A894B895C89CA01B9010E9487
:1001E0009305DC01CB01BC01CD0120E030E040E013
:1001F00054E40E94BA06DC01CB018D839E83AF8359
:10020000B8871A82198248C08D859E85AF85B889C6
:10021000BC01CD010E94A809DC01CB01BC01CD01CC
:1002200020E030E04EEF52E40E94C005DC01CB013B
:1002300089879A87AB87BC876D857E858F859889EE
:100240002D813E814F8158850E949305DC01CB01B1
:100250008D879E87AF87B88B69857A858B859C85CE
:1002600020E030E040E053E40E949305DC01CB0144
:10027000BC01CD010E946607DC01CB019C838B830E
:1002800089819A812B81FC01EE5DFE4F208389815B
:100290009A8101969A83898389819A8122E08030AC
:1002A00092070CF4B1CF64960FB6F894DEBF0FBE80
:1002B000CDBFCF91DF910895DF93CF9300D0CDB71D
:1002C000DEB70E94CF0086E293E040E052EC61E0AE
:1002D00070E00E94CB01A4E2B0E0E4E2F0E08081B3
:1002E00080628C93E5E2F0E080E28083A1E8B0E0F8
:1002F000E1E8F0E0808188608C93AFE6B0E0EFE663
:10030000F0E0808182608C93E8E8F0E086E891E09C
:1003100091838083789486E293E00E94C8011A82D8
:100320001816190614F481E08A838A81882399F3C8
:10033000A5E2B0E0E5E2F0E0908180E289278C93CD
:1003400086E293E00E94C50189838981813619F78D
:1003500086E293E020E031E0B9010E941F02A1E8AB
:10036000B0E0E1E8F0E0808185608C93D4CF87E154
:1003700091E090932703809326030895862F0E948F
:10038000980308950E94D00308950E94B103089530
:100390000E94A0030895CB01BA010E945F03089553
:1003A000DC01ED91FC910190F081E02D099508951B
:1003B000DC01ED91FC910190F081E02D099508950B
:1003C0000F931F93CF93DF938C01EB0109C021960C
:1003D000D801ED91FC910190F081E02DC8010995C3
:1003E00068816623A1F7DF91CF911F910F91089546
:1003F0000F931F938C01DC01ED91FC910190F08132
:10040000E02D6DE00995D801ED91FC910190F0810E
:10041000E02D6AE0C80109951F910F9108950F938F
:100420001F938C01DC01ED91FC910190F081E02D96
:100430000995C8010E94F8011F910F9108950F932B
:100440001F938C010E94E001C8010E94F8011F91D6
:100450000F9108950F931F938C01DC01ED91FC9196
:100460000190F081E02D0995C8010E94F8011F91CB
:100470000F9108952F923F924F925F926F927F92C9
:100480008F929F92AF92BF92CF92DF92EF92FF92A4
:100490000F931F93DF93CF93CDB7DEB7A0970FB61F
:1004A000F894DEBF0FBECDBF1C016A017B01411570
:1004B00051056105710549F4DC01ED91FC91019054
:1004C000F081E02D60E3099554C0882499245401FB
:1004D000422E55246624772401E010E00C0F1D1FE6
:1004E000080D191DC701B601A30192010E941A0946
:1004F000F80160830894811C911CA11CB11CC701E8
:10050000B601A30192010E941A09C901DA016C0126
:100510007D01C114D104E104F104F1F681E0E82E7B
:10052000F12CEC0EFD1EE80CF91C3E010894611C38
:10053000711CD501C4010197A109B1096C01C8184A
:10054000D90814C0F601EE0DFF1D60816A3010F469
:10055000605D01C0695CD101ED91FC910190F08179
:10056000E02DC10109950894E108F1086E147F049B
:1005700049F7A0960FB6F894DEBF0FBECDBFCF915E
:10058000DF911F910F91FF90EF90DF90CF90BF9080
:10059000AF909F908F907F906F905F904F903F9023
:1005A0002F9008952AE00E943A0208950F931F9316
:1005B0008C010E94D202C8010E94F8011F910F9184
:1005C0000895AB0160E070E00E94D20208950F939D
:1005D0001F938C01AB0160E070E00E94D202C80161
:1005E0000E94F8011F910F910895EF92FF920F93CF
:1005F0001F93CF93DF93EC017A018B0177FF0FC03C
:10060000E881F9810190F081E02D6DE20995109566
:100610000095F094E094E11CF11C011D111D2AE0ED
:10062000B801A701CE010E943A02DF91CF911F913C
:100630000F91FF90EF9008950F931F938C010E94EC
:10064000F502C8010E94F8011F910F910895AB01B6
:10065000662757FD6095762F0E94F50208950F9347
:100660001F938C01AB01662757FD6095762F0E9482
:10067000F502C8010E94F8011F910F910895DC0155
:100680002115310541F4ED91FC910190F081E02DAF
:10069000642F099508952A30310519F40E94F50256
:1006A00008950E943A0208950F931F938C010E94AF
:1006B0003F03C8010E94F8011F910F910895EF9226
:1006C000FF920F931F937B018C0122E030E040E00A
:1006D00050E00E943C09205C3D4B404F5F4FCA01F7
:1006E000B901A80197010E943C09C901DA010197EB
:1006F000A109B109292F3A2F4B2F552747FD5A95AC
:100700000196A11DB11D2093C50081508093C400A6
:10071000E1ECF0E08081806180838081886080836B
:100720008081806880831F910F91FF90EF900895E2
:10073000982F8091C00085FFFCCF9093C60008954C
:10074000809128039091290380589F4F20912A037C
:1007500030912B03821B930B60E870E00E94070925
:10076000089540912A0350912B0380912803909182
:1007700029038417950719F42FEF3FEF0FC0FA01F3
:10078000E45DFC4F2081CA01019660E870E00E94A0
:10079000070990932B0380932A0330E0C901089541
:1007A00080912A0390912B0390932903809328032F
:1007B00008951F920F920FB60F9211242F933F931B
:1007C0004F935F936F937F938F939F93AF93BF9359
:1007D000EF93FF934091C600E0912803F091290325
:1007E000CF01019660E870E00E9407099C018091AA
:1007F0002A0390912B032817390739F0E45DFC4F49
:1008000040833093290320932803FF91EF91BF91F8
:10081000AF919F918F917F916F915F914F913F9198
:100820002F910F900FBE0F901F901895A0E0B0E091
:10083000ECE1F4E00C946B09DC012B01FA019C91D2
:10084000923008F439C1EB018881823008F433C159
:10085000943069F4843009F02FC111969C9111975E
:100860008981981709F428C1A9E1B1E025C1843034
:1008700009F421C18230A9F4923009F01DC19A0116
:10088000AD0188E0EA010990AE01E90109929E01FB
:100890008150C1F7E201898111969C91892381835E
:1008A00008C1923009F407C112962D903C9013971D
:1008B000EB018A819B811496AD90BD90CD90DC9028
:1008C0001797EC80FD800E811F819101281B390B49
:1008D000B90137FF04C066277727621B730B6032AC
:1008E00071050CF061C0121613066CF53701480152
:1008F000062E04C096948794779467940A94D2F74E
:1009000021E030E040E050E004C0220F331F441FDC
:10091000551F6A95D2F721503040404050402E215B
:100920003F2140235123211531054105510521F077
:1009300021E030E040E050E079018A01E628F72824
:10094000082919293CC0232BD1F1260E371E350169
:100950004601062E04C096948794779467940A946F
:10096000D2F721E030E040E050E004C0220F331F16
:10097000441F551F6A95D2F72150304040405040E7
:100980002A213B214C215D212115310541055105CD
:1009900021F021E030E040E050E059016A01A62852
:1009A000B728C828D9280BC0821593052CF01C0144
:1009B000AA24BB24650103C0EE24FF2487011196FD
:1009C0009C91D20111968C91981709F445C09923F6
:1009D00039F0A80197012A193B094C095D0906C0A5
:1009E000A60195012E193F09400B510B57FD08C078
:1009F00011823382228224833583468357831DC02C
:100A000081E081833382228288279927DC01821B3F
:100A1000930BA40BB50B84839583A683B7830DC07A
:100A2000220F331F441F551F24833583468357836A
:100A300082819381019793838283248135814681CA
:100A40005781DA01C9010197A109B1098F5F9F4F51
:100A5000AF4FBF4328F30BC0918333822282EA0C4D
:100A6000FB1C0C1D1D1DE482F5820683178383E0A9
:100A70008083248135814681578157FF1AC0C9017F
:100A8000AA2797FDA095BA2F81709070A070B070C2
:100A90005695479537952795822B932BA42BB52BED
:100AA00084839583A683B783828193810196938300
:100AB0008283DF0101C0D201CD01CDB7DEB7E2E113
:100AC0000C948709A0E2B0E0E8E6F5E00C94770921
:100AD00069837A838B839C832D833E834F835887DE
:100AE000E9E0EE2EF12CEC0EFD1ECE010196B701D1
:100AF0000E948F088E010F5E1F4FCE010596B80130
:100B00000E948F088A8991E089278A8BC701B801E2
:100B1000AE01475E5F4F0E9416040E94BA07A0967E
:100B2000E6E00C949309A0E2B0E0E9E9F5E00C946A
:100B3000770969837A838B839C832D833E834F83DC
:100B40005887F9E0EF2EF12CEC0EFD1ECE01019638
:100B5000B7010E948F088E010F5E1F4FCE010596D0
:100B6000B8010E948F08C701B801AE01475E5F4F10
:100B70000E9416040E94BA07A096E6E00C9493091E
:100B8000A0E2B0E0E6ECF5E00C946B0969837A83AF
:100B90008B839C832D833E834F835887CE010196A0
:100BA000BE01675F7F4F0E948F08CE010596BE0190
:100BB0006F5E7F4F0E948F089985923088F08989F7
:100BC0008230C8F0943019F4823051F404C084307B
:100BD00029F4923081F489E191E0C6C0923049F461
:100BE00020E09A858A89981321E02A87CE01099608
:100BF000BBC0823049F420E09A858A89981321E0AD
:100C00002A8BCE014196B0C02D843E844F845888F3
:100C10006D887E888F88988CEE24FF248701AA2413
:100C2000BB24650140E050E060E070E0E0E0F0E00F
:100C3000C10181709070892BE9F0E60CF71C081D4A
:100C4000191D9A01AB012A0D3B1D4C1D5D1D80E055
:100C500090E0A0E0B0E0E614F7040805190520F4E0
:100C600081E090E0A0E0B0E0BA01A901480F591F6F
:100C70006A1F7B1FAA0CBB1CCC1CDD1C97FE08C086
:100C800081E090E0A0E0B0E0A82AB92ACA2ADB2AD5
:100C90003196E032F10549F0660C771C881C991CEE
:100CA0005694479437942794C3CFFA85EA892B89C1
:100CB0003C898B859C85280F391F2E5F3F4F17C0BD
:100CC000CA0181709070892B61F016950795F79491
:100CD000E79480E090E0A0E0B0E8E82AF92A0A2B47
:100CE0001B2B76956795579547952F5F3F4F77FD5F
:100CF000E7CF0CC0440F551F661F771F17FD4160DB
:100D0000EE0CFF1C001F111F21503040403090E0BE
:100D1000590790E0690790E4790760F32B8F3C8FC7
:100D2000DB01CA018F779070A070B070803491059C
:100D3000A105B10561F447FD0AC0E114F104010504
:100D4000110529F0405C5F4F6F4F7F4F40781A8E3E
:100D5000FE1711F081E08A8F4D8F5E8F6F8F78A321
:100D600083E0898FCE0149960E94BA07A096E2E1FE
:100D70000C948709A8E1B0E0E0ECF6E00C9473096C
:100D800069837A838B839C832D833E834F8358872B
:100D9000B9E0EB2EF12CEC0EFD1ECE010196B70151
:100DA0000E948F088E010F5E1F4FCE010596B8017D
:100DB0000E948F082985223008F47EC0398932309C
:100DC00010F4B8017CC08A859A8989278A872430E3
:100DD00011F0223031F4231709F06EC069E171E09F
:100DE0006EC0343039F41D861E861F86188A1C8614
:100DF0001B8604C0323021F484E08987B7015FC0CC
:100E00002B853C858B899C89281B390B3C872B873C
:100E1000ED84FE840F851889AD88BE88CF88D88C74
:100E2000EA14FB040C051D0540F4EE0CFF1C001F2A
:100E3000111F215030403C872B8720E030E040E0FC
:100E400050E080E090E0A0E0B0E460E070E0EA1400
:100E5000FB040C051D0540F0282B392B4A2B5B2B7E
:100E6000EA18FB080C091D09B695A7959795879573
:100E7000EE0CFF1C001F111F6F5F7F4F6F3171055C
:100E800031F7DA01C9018F779070A070B0708034AB
:100E90009105A105B10561F427FD0AC0E114F10433
:100EA0000105110529F0205C3F4F4F4F5F4F20781F
:100EB0002D873E874F87588BBE01675F7F4FCB01E1
:100EC0000E94BA076896EAE00C948F09ACE0B0E0A3
:100ED000ECE6F7E00C947B0969837A838B839C832F
:100EE000CE010196BE016B5F7F4F0E948F088D81FE
:100EF000823061F1823050F1843021F48E81882378
:100F000051F12EC02F81388537FD20C06E812F31E1
:100F100031051CF06623F9F023C08EE190E0821BBE
:100F2000930B29853A854B855C8504C0569547957A
:100F3000379527958A95D2F76623B1F0509540955D
:100F4000309521953F4F4F4F5F4F0EC020E030E06E
:100F500040E050E009C02FEF3FEF4FEF5FE704C0E4
:100F600020E030E040E050E8B901CA012C96E2E010
:100F70000C949709DF92EF92FF920F931F93FC015D
:100F8000E480F58006811781D1808081823048F429
:100F900080E090E0A0E1B0E0E82AF92A0A2B1B2BC0
:100FA000A5C0843009F49FC0823021F4EE24FF24D0
:100FB000870105C0E114F1040105110519F4E0E011
:100FC000F0E096C0628173819FEF623879070CF080
:100FD0005BC022E83FEF261B370B2A3131052CF08E
:100FE00020E030E040E050E02AC0B801A701022E26
:100FF00004C076956795579547950A94D2F781E096
:1010000090E0A0E0B0E004C0880F991FAA1FBB1FAA
:101010002A95D2F70197A109B1098E219F21A0231A
:10102000B1230097A105B10521F081E090E0A0E097
:10103000B0E09A01AB01282B392B4A2B5B2BDA014C
:10104000C9018F779070A070B07080349105A105B0
:10105000B10539F427FF09C0205C3F4F4F4F5F4F68
:1010600004C0215C3F4F4F4F5F4FE0E0F0E0203085
:10107000A0E03A07A0E04A07A0E45A0710F0E1E038
:10108000F0E079018A0127C06038710564F5FB0141
:10109000E158FF4FD801C7018F779070A070B070F2
:1010A00080349105A105B10539F4E7FE0DC080E457
:1010B00090E0A0E0B0E004C08FE390E0A0E0B0E0FA
:1010C000E80EF91E0A1F1B1F17FF05C0169507958E
:1010D000F794E794319687E016950795F794E7948F
:1010E0008A95D1F705C0EE24FF248701EFEFF0E0E9
:1010F0006E2F679566276795902F9F77D794DD248D
:10110000D7948E2F8695492F462B582F5D29B701EE
:10111000CA011F910F91FF90EF90DF900895FC019D
:10112000DB01408151812281622F6F7770E0221FA5
:101130002227221F9381892F880F822B282F30E0AE
:10114000991F9927991F11969C9311972115310585
:10115000A9F5411551056105710511F482E037C00B
:1011600082E89FEF13969C938E9312979A01AB019E
:1011700067E0220F331F441F551F6A95D1F783E0A4
:101180008C930DC0220F331F441F551F12968D9153
:101190009C911397019713969C938E9312972030EE
:1011A00080E0380780E0480780E4580758F3149639
:1011B0002D933D934D935C93179708952F3F3105E1
:1011C00079F4411551056105710519F484E08C939A
:1011D000089564FF03C081E08C9312C01C9210C07C
:1011E0002F57304013963C932E93129783E08C93A5
:1011F00087E0440F551F661F771F8A95D1F77064EB
:1012000014964D935D936D937C931797089597FB78
:10121000092E07260AD077FD04D049D006D0002039
:101220001AF4709561957F4F0895F6F79095819522
:101230009F4F0895A1E21A2EAA1BBB1BFD010DC0F2
:10124000AA1FBB1FEE1FFF1FA217B307E407F50776
:1012500020F0A21BB30BE40BF50B661F771F881F52
:10126000991F1A9469F760957095809590959B01E8
:10127000AC01BD01CF01089597FB092E05260ED0C4
:1012800057FD04D0D7DF0AD0001C38F450954095A4
:10129000309521953F4F4F4F5F4F0895F6F790954A
:1012A0008095709561957F4F8F4F9F4F0895AA1B32
:1012B000BB1B51E107C0AA1FBB1FA617B70710F041
:1012C000A61BB70B881F991F5A95A9F78095909573
:1012D000BC01CD0108952F923F924F925F926F9281
:1012E0007F928F929F92AF92BF92CF92DF92EF92B6
:1012F000FF920F931F93CF93DF93CDB7DEB7CA1B37
:10130000DB0B0FB6F894DEBF0FBECDBF09942A8861
:10131000398848885F846E847D848C849B84AA8409
:10132000B984C884DF80EE80FD800C811B81AA8196
:10133000B981CE0FD11D0FB6F894DEBF0FBECDBF61
:10134000ED010895EE0FFF1F0590F491E02D099433
:101350009F9305D00F9007FCEE5F28C0CEC03FD012
:10136000E8F3E894E0E0BB279F57F0F02AED3FE078
:1013700049EC06C0EE0FBB0F661F771F881F28F0D1
:10138000B23A62077307840728F0B25A620B730BF4
:10139000840BE3959A9572F7803830F49A95BB0FD9
:1013A000661F771F881FD2F790489BC0EF93E0FF1E
:1013B00006C0A2EA2AED3FE049EC5FEB37D0BFD090
:1013C0000F90039401FC9058E8E6F0E099C057FDB7
:1013D0009058440F551F59F05F3F71F04795880FA3
:1013E00097FB991F61F09F3F79F08795089512163A
:1013F00013061406551FF2CF4695F1DF08C01616E6
:1014000017061806991FF1CF869571056105089496
:10141000089587D030F08CD020F031F49F3F11F444
:101420001EF46BC00EF4E095E7FB53C0E92FCFDF4D
:1014300080F3BA17620773078407950718F071F4F1
:101440009EF58EC00EF4E0950B2EBA2FA02D0B0149
:10145000B90190010C01CA01A0011124FF27591BF9
:1014600099F0593F50F4503E68F11A16F040A22FFF
:10147000232F342F4427585FF3CF46953795279570
:10148000A795F0405395C9F77EF41F16BA0B620B6F
:10149000730B840BBAF09150A1F0FF0FBB1F661FB6
:1014A000771F881FC2F70EC0BA0F621F731F841FF9
:1014B00048F4879577956795B795F7959E3F08F01F
:1014C000B3CF9395880F08F09927EE0F97958795DE
:1014D000089597F99F6780E870E060E008959F3F66
:1014E00031F0915020F4879577956795B795880FDF
:1014F000911D9695879597F908959FEF80EC089533
:101500009F938F937F936F93FF93EF939B01AC0116
:1015100037DBEF91FF912BD02F913F914F915F914E
:101520002FCB00240A9416161706180609060895EC
:1015300000240A9412161306140605060895092EAF
:101540000394000C11F4882352F0BB0F40F4BF2B1E
:1015500011F460FF04C06F5F7F4F8F4F9F4F08955E
:10156000E894BB2766277727CB0197F90895DF9387
:10157000CF931F930F93FF92EF92DF927B018C0129
:10158000689405C0DA2EEF0121D0FE01E894A59100
:101590002591359145915591AEF3EF0147DFFE015D
:1015A0009701A801DA9479F7DF90EF90FF900F91FF
:1015B0001F91CF91DF910895B4DF28F0B9DF18F0C3
:1015C000952309F086CF99CF1124CBCF00DFA0F36C
:1015D000959FD1F3950F50E0551F629FF001729FC8
:1015E000BB27F00DB11D639FAA27F00DB11DAA1FE7
:1015F000649F6627B00DA11D661F829F2227B00D34
:10160000A11D621F739FB00DA11D621F839FA00DBE
:10161000611D221F749F3327A00D611D231F849F0E
:10162000600D211D822F762F6A2F11249F57504065
:101630008AF0E1F088234AF0EE0FFF1FBB1F661F00
:10164000771F881F91505040A9F79E3F510570F0B9
:1016500040CF87CF5F3FECF3983EDCF386957795DC
:101660006795B795F795E7959F5FC1F7FE2B880FB4
:0E167000911D9695879597F90895F894FFCFF0
:10167E0057656C636F6D6520746F20656C65637460
:10168E0069630000000000BE0100000000000000C1
:02169E0000004A
:00000001FF
